** EXPERIMENTAL (HLL) ** Open Watcom Linker Version 1.6beta1 Limited Availability
Portions Copyright (c) 1985-2002 Sybase, Inc. All Rights Reserved.
Created on:       13/11/17 16:25:02
Warning! W1121: file U:/tmp\ldconv_readline_obj_19c252885a341cfc38.obj(U:\DEV\python-2.7.5\Modules\readline.c): '_initreadline' has already been exported
Executable Image: build/lib.os2knix-2.7/readline.pyd
creating an OS/2 EMX dynamic link library


                        +------------+
                        |   Groups   |
                        +------------+

Group                           Address              Size
=====                           =======              ====

CGROUP                          0001:00000000        00036e80
DGROUP                          0002:00000000        00005930



                        +--------------+
                        |   Segments   |
                        +--------------+

Segment                Class          Group          Address         Size
=======                =====          =====          =======         ====

TEXT32                 CODE           CGROUP         0001:00000000   00036e80
________TEXT           CODE           CGROUP         0001:00036e80   00000000
DATA32                 DATA           DGROUP         0002:00000000   00003ec0
SET1__os2dll           DATA           DGROUP         0002:00003ec0   00000004
SET2__os2dll           DATA           DGROUP         0002:00003ec4   00000000
SET3__os2dll           DATA           DGROUP         0002:00003ec4   00000004
SET1___CTOR_LIST__     DATA           DGROUP         0002:00003ec8   00000004
SET2___CTOR_LIST__     DATA           DGROUP         0002:00003ecc   00000000
SET3___CTOR_LIST__     DATA           DGROUP         0002:00003ecc   00000004
SET1___DTOR_LIST__     DATA           DGROUP         0002:00003ed0   00000004
SET2___DTOR_LIST__     DATA           DGROUP         0002:00003ed4   00000000
SET3___DTOR_LIST__     DATA           DGROUP         0002:00003ed4   00000004
SET1___crtinit1__      DATA           DGROUP         0002:00003ed8   00000004
SET2___crtinit1__      DATA           DGROUP         0002:00003edc   00000000
SET3___crtinit1__      DATA           DGROUP         0002:00003edc   00000004
SET1___crtexit1__      DATA           DGROUP         0002:00003ee0   00000004
SET2___crtexit1__      DATA           DGROUP         0002:00003ee4   00000000
SET3___crtexit1__      DATA           DGROUP         0002:00003ee4   00000004
SET1___eh_frame__      DATA           DGROUP         0002:00003ee8   00000004
SET2___eh_frame__      DATA           DGROUP         0002:00003eec   00000008
SET3___eh_frame__      DATA           DGROUP         0002:00003ef4   00000004
SET1___eh_init__       DATA           DGROUP         0002:00003ef8   00000004
SET2___eh_init__       DATA           DGROUP         0002:00003efc   00000004
SET3___eh_init__       DATA           DGROUP         0002:00003f00   00000004
SET1___eh_term__       DATA           DGROUP         0002:00003f04   00000004
SET2___eh_term__       DATA           DGROUP         0002:00003f08   00000004
SET3___eh_term__       DATA           DGROUP         0002:00003f0c   00000004
SET1___fork_parent1__  DATA           DGROUP         0002:00003f10   00000004
SET2___fork_parent1__  DATA           DGROUP         0002:00003f14   00000000
SET3___fork_parent1__  DATA           DGROUP         0002:00003f14   00000004
SET1___fork_child1__   DATA           DGROUP         0002:00003f18   00000004
SET2___fork_child1__   DATA           DGROUP         0002:00003f1c   00000000
SET3___fork_child1__   DATA           DGROUP         0002:00003f1c   00000004
________DATA           DATA           DGROUP         0002:00003f20   00000000
BSS32                  BSS            DGROUP         0002:00003f20   000016f0
c_common               BSS            DGROUP         0002:00005610   00000320
________BSS            BSS            DGROUP         0002:00005930   00000000


                        +----------------+
                        |   Memory Map   |
                        +----------------+

* = unreferenced symbol
+ = symbol only referenced locally

Address        Symbol
=======        ======

Module: U:\usr\lib\dll0hi.obj({standard input})
0001:00000000* __text
0002:00000000* __data
0002:00000000* ___data_start
0002:00003f20* ___bss_start
0002:00003ec0+ __os2dll
0002:00003ec8  ___CTOR_LIST__
0002:00003ed0  ___DTOR_LIST__
0002:00003ed8* ___crtinit1__
0002:00003ee0* ___crtexit1__
0002:00003ee8  ___eh_frame__
0002:00003ef8  ___eh_init__
0002:00003f04  ___eh_term__
0002:00003f10+ ___fork_parent1__
0002:00003f18+ ___fork_child1__
Module: U:/tmp\ldconv_readline_obj_19c252885a341cfc38.obj(U:\DEV\python-2.7.5\Modules\readline.c)
0001:00000f32  _initreadline
Module: U:\usr\local473\lib\libc_dll.lib(dllinit.obj)
0001:00001250  _DLL_InitTerm
Module: U:\usr\lib\libend.lib(src/libend/386/endlink386.asm)
0002:00005930  _end
0002:00003f20  _edata
Module: U:\usr\lib\libend.lib(src/libend/386/end.asm)
0001:00036e80* _etext
0001:00036e80* __etext
0000:00000000  WEAK$ZERO
0002:00005930  __end
0002:00003f20  __edata
Module: U:\extras\lib\libreadline.lib(history.obj)
0002:00005610  _history_offset
0002:00005620  _history_length
0002:00005630  _history_max_entries
0002:00005640+ _max_input_history
0001:000012b0* _history_set_history_state
0001:000012eb  _using_history
0001:000012fa  _where_history
0001:00001304  _history_set_pos
0001:00001330  _history_list
0001:0000133a  _current_history
0001:0000135d  _previous_history
0001:0000137f  _next_history
0001:000013a5  _history_get
0001:000013ce  _replace_history_data
0001:00001466  _remove_history
0001:000014b7* _unstifle_history
0001:000014de  _history_is_stifled
0001:000014e8  _history_get_history_state
0001:00001537* _history_total_bytes
0001:000015b9  _replace_history_entry
0001:00001662* _alloc_history_entry
0001:000016bc* _copy_history_entry
0001:00001723  _add_history_time
0001:0000177d  _free_history_entry
0001:000017bf  _clear_history
0001:0000181a  _stifle_history
0001:000018db  _add_history
0001:00001a42* _history_get_time
0002:00000db0  _history_base
Module: U:\extras\lib\libreadline.lib(complete.obj)
0002:00005650+ _rl_completion_found_quote
0002:00005660+ _rl_completion_quote_character
0002:00005670+ _rl_completion_mark_symlink_dirs
0002:00005680  __rl_print_completions_horizontally
0002:00005690+ _rl_completion_invoking_key
0002:000056a0  _rl_inhibit_completion
0001:00001a80* _rl_completion_mode
0001:00001abf  __rl_reset_completion_state
0001:00001b2f* __rl_free_match_list
0001:0000268e* __rl_find_completion_word
0001:00002e2d* _rl_filename_completion_function
0001:0000360e* _rl_username_completion_function
0001:00003740  _rl_completion_matches
0001:000038f9* _rl_display_match_list
0001:00003e6a  _rl_menu_complete
0001:00004386  _rl_backward_menu_complete
0001:0000439a  _rl_old_menu_complete
0001:0000470b  _rl_complete_internal
0001:00004bea  _rl_insert_completions
0001:00004c05  _rl_possible_completions
0001:00004c20  _rl_complete
0002:00000de0* _rl_filename_quoting_desired
0002:00000ddc* _rl_ignore_completion_duplicates
0002:00000dec* _rl_sort_completion_matches
0002:00000dc0  __rl_complete_mark_directories
0002:00000dd8  _rl_basic_quote_characters
0002:00000de4* _rl_filename_quoting_function
0002:00000de8  _rl_completion_append_character
0002:00000dc4  __rl_match_hidden_files
0002:00000dc8  __rl_completion_columns
0002:00000dd0  __rl_page_completions
0002:00000dcc  _rl_completion_query_items
0002:00000dd4  _rl_basic_word_break_characters
0002:00003ff4  __rl_complete_show_all
0002:00003ff8  __rl_complete_show_unmodified
0002:00004044* _rl_completer_quote_characters
0002:00004000  __rl_completion_case_fold
0002:00004050* _rl_filename_completion_desired
0002:00004058* _rl_filename_dequoting_function
0002:00004054* _rl_ignore_some_completions_function
0002:0000400c  _rl_visible_stats
0002:00004018* _rl_directory_completion_hook
0002:00004040* _rl_completion_word_break_hook
0002:0000405c* _rl_char_is_quoted_p
0002:0000404c* _rl_special_prefixes
0002:0000403c  _rl_completer_word_break_characters
0002:00004048* _rl_filename_quote_characters
0002:00004010  __rl_skip_completed_text
0002:00004060  _rl_completion_suppress_append
0002:00004064* _rl_completion_suppress_quote
0002:0000401c* _rl_directory_rewrite_hook
0002:00004020* _rl_filename_rewrite_hook
0002:00004024  _rl_complete_with_tilde_expansion
0002:00004004  __rl_completion_case_map
0002:00004030  _rl_attempted_completion_function
0002:00004034  _rl_attempted_completion_over
0002:00004008  __rl_completion_prefix_display_length
0002:00003ff0  _rl_completion_display_matches_hook
0002:00004038  _rl_completion_type
0002:00003ffc  __rl_complete_mark_symlink_dirs
0002:0000402c* _rl_menu_completion_entry_function
0002:00004014  __rl_menu_complete_prefix_first
0002:00004028* _rl_completion_entry_function
Module: U:\extras\lib\libreadline.lib(readline.obj)
0002:000056b0  _rl_mark
0002:000056c0  _rl_end
0002:000056d0  _rl_point
0002:000056e0  _rl_done
0002:000056f0+ __rl_in_stream
0002:00005700  __rl_out_stream
0002:00005710+ _rl_executing_keymap
0002:00005720  _rl_dispatching
0002:00005730+ __rl_dispatching_keymap
0002:00005740+ _rl_num_chars_to_read
0002:00005750  __rl_top_level
0002:00005790  __rl_comment_begin
0001:00004cb0  __rl_init_line_state
0001:00004ce0  __rl_set_the_line
0001:00004cef* _rl_save_state
0001:00004da5* _rl_restore_state
0001:00004e60* __rl_keyseq_cxt_alloc
0001:00004fe4  _rl_initialize
0001:00005215* __rl_keyseq_cxt_dispose
0001:00005221* __rl_keyseq_chain_dispose
0001:0000524c* __rl_dispatch_subseq
0001:0000564c  __rl_dispatch
0001:00005782  __rl_dispatch_callback
0001:0000588a  __rl_internal_char_cleanup
0001:00005945  _readline_internal_char
0001:00005abf  _readline_internal_teardown
0001:00005be5  _readline_internal_setup
0001:00005cdb  _rl_set_prompt
0001:00005d56  _readline
0002:00000dfc  __rl_keymap
0002:00000e04  _rl_insert_mode
0002:00000e00  _rl_editing_mode
0002:00000e1c  __rl_bind_stty_chars
0002:00000e18  __rl_convert_meta_chars_to_ascii
0002:00000e0c  _rl_arg_sign
0002:00000e08  _rl_numeric_arg
0002:00000e10  __rl_eof_char
0002:00000df0* _rl_library_version
0002:00000df4* _rl_readline_version
0002:00000df8* _rl_gnu_readline_p
0002:00000e14  __rl_bell_preference
0002:00000e20  __rl_echo_control_chars
0002:00004298  _rl_line_buffer
0002:0000429c  _rl_line_buffer_len
0002:0000426c  _rl_prompt
0002:00004258  _rl_readline_state
0002:0000425c  _rl_last_func
0002:00004278  _rl_key_sequence_length
0002:00004260  _rl_instream
0002:00004264  _rl_outstream
0002:00004284  _rl_pending_input
0002:000042a0  __rl_kscxt
0002:000042a4  __rl_parsing_conditionalized_out
0002:00004288  _rl_terminal_name
0002:0000428c  __rl_horizontal_scroll_mode
0002:00004294  _rl_erase_empty_line
0002:00004250  __rl_last_command_was_kill
0002:000042ac  __rl_revert_all_at_newline
0002:0000427c  _rl_startup_hook
0002:00004268  __rl_echoing_p
0002:00004274* _rl_already_prompted
0002:00004280  _rl_pre_input_hook
0002:00004270  _rl_visible_prompt_length
0002:000042b0  __rl_meta_flag
0002:00004254  _rl_explicit_arg
0002:00004290  __rl_mark_modified_lines
0002:000042a8  __rl_output_meta_chars
Module: U:\extras\lib\libreadline.lib(display.obj)
0001:00005df0  _rl_on_new_line
0001:00005e4b  _rl_forced_update_display
0001:00005e7f  _rl_character_len
0001:00005eed  _rl_reset_line_state
0001:00005f18  _rl_save_prompt
0001:00005fbd  __rl_current_display_line
0001:00006001  __rl_clear_screen
0001:00006030  __rl_clear_to_eol
0001:00006095  __rl_erase_entire_line
0001:0000610c  __rl_move_vert
0001:000061c8  __rl_clean_up_for_exit
0001:0000642e  __rl_strip_prompt
0001:00006451  __rl_make_prompt_for_search
0001:00006545  __rl_erase_at_end_of_line
0001:000065c1  __rl_move_cursor_relative
0001:000066cf  __rl_update_final
0001:000067ae  _rl_restore_prompt
0001:00006878  __rl_redisplay_after_sigwinch
0001:00006a00  _rl_clear_message
0001:00006a32  _rl_expand_prompt
0001:00006baf  _rl_message
0001:00006c5f* _rl_show_char
0001:00006f0a  _rl_on_new_line_with_prompt
0001:00007990  _rl_redisplay
0002:00000e30  _rl_redisplay_function
0002:00004314* __rl_last_v_pos
0002:00004310  __rl_last_c_pos
0002:00004318  __rl_vis_botlin
0002:0000430c  _rl_display_prompt
0002:00004300  _rl_display_fixed
0002:00004304* __rl_suppress_redisplay
0002:00004308  __rl_want_redisplay
Module: U:\extras\lib\libreadline.lib(text.obj)
0001:00008890  __rl_fix_point
0001:000088e5* __rl_forward_char_internal
0001:000088ff  _rl_beg_of_line
0001:00008910  _rl_end_of_line
0001:00008921  _rl_do_lowercase_version
0001:00008928  __rl_set_mark_at_pos
0001:00008945  _rl_set_mark
0001:00008972  _rl_exchange_point_and_mark
0001:000089b5  __rl_char_search_internal
0001:00008ab2  _rl_backward_byte
0001:00008b06  _rl_forward_byte
0001:00008b8c  _rl_forward_char
0001:00008b98* _rl_forward
0001:00008ba4  _rl_backward_char
0001:00008bb0* _rl_backward
0001:00008c1f  _rl_backward_char_search
0001:00008c95  _rl_char_search
0001:00008ce0  _rl_skip_csi_sequence
0001:00008d05  _rl_backward_word
0001:00008dad  _rl_forward_word
0001:00008fed  _rl_capitalize_word
0001:00009001  _rl_downcase_word
0001:00009015  _rl_upcase_word
0001:00009029  _rl_newline
0001:000090c2  _rl_arrow_keys
0001:00009185  _rl_refresh_line
0001:000091cc  _rl_clear_screen
0001:0000920a  _rl_replace_line
0001:0000926e  _rl_delete_text
0001:0000934d  _rl_delete_horizontal_space
0001:00009425  _rl_delete
0001:000094ad  __rl_rubout_char
0001:0000958c  _rl_delete_or_show_completions
0001:000095bb  _rl_rubout_or_delete
0001:000095ea  _rl_insert_text
0001:00009731  _rl_transpose_chars
0001:000097cd  _rl_transpose_words
0001:000098fd  _rl_insert_comment
0001:000099a2  __rl_insert_char
0001:00009a9a* __rl_overwrite_rubout
0001:00009b8d  _rl_rubout
0001:00009be0  _rl_tab_insert
0001:00009c46  _rl_quoted_insert
0001:00009cb7  __rl_overwrite_char
0001:00009d1d  _rl_insert
0001:00009d44  __rl_replace_text
Module: U:\extras\lib\libreadline.lib(bind.obj)
0002:000057a0+ _rl_binding_keymap
0001:00009da0  _rl_bind_key
0001:00009e01  _rl_bind_key_in_map
0001:00009e34* _rl_unbind_key
0001:00009e4f* _rl_unbind_key_in_map
0001:00009e71* _rl_unbind_function_in_map
0001:00009eb3* _rl_untranslate_keyseq
0001:0000a0c6* _rl_function_of_keyseq
0001:0000a1ba* _rl_get_keymap_name
0001:0000a1ee* _rl_set_keymap
0001:0000a1ff* _rl_get_keymap
0001:0000a209  _rl_set_keymap_from_edit_mode
0001:0000a240* _rl_get_keymap_name_from_edit_mode
0001:0000a8f8* _rl_macro_dumper
0001:0000a912  _rl_dump_macros
0001:0000ab78* _rl_get_keymap_by_name
0001:0000aee9* _rl_variable_dumper
0001:0000aff1  _rl_dump_variables
0001:0000b03b* _rl_variable_value
0001:0000b0ef* _rl_list_funmap_names
0001:0000b142* _rl_invoking_keyseqs_in_map
0001:0000b44a* _rl_invoking_keyseqs
0001:0000b48f* _rl_variable_bind
0001:0000b94a* _rl_named_function
0001:0000b9f9* _rl_function_dumper
0001:0000bbc1  _rl_dump_functions
0001:0000bc0b* _rl_unbind_command_in_map
0001:0000bc68* _rl_translate_keyseq
0001:0000c333* _rl_generic_bind
0001:0000c522* _rl_macro_bind
0001:0000c597* _rl_set_key
0001:0000c5c0  _rl_bind_keyseq_in_map
0001:0000c5e9* _rl_bind_keyseq_if_unbound_in_map
0001:0000c64b  _rl_bind_keyseq_if_unbound
0001:0000c66e* _rl_bind_key_if_unbound
0001:0000c69b* _rl_bind_key_if_unbound_in_map
0001:0000c6c6* _rl_bind_keyseq
0001:0000c746  _rl_parse_and_bind
0001:0000d340* __rl_possible_control_prefixes
0001:0000d354* __rl_possible_meta_prefixes
0001:0000d26e  _rl_read_init_file
0001:0000d2be  _rl_re_read_init_file
0001:0000d2f7* _rl_add_defun
0002:00000e40  _rl_readline_name
Module: U:\extras\lib\libreadline.lib(input.obj)
0001:0000d8e0  __rl_any_typein
0001:0000d8f6  __rl_unget_char
0001:0000d959  __rl_pushed_input_available
0001:0000d96f* _rl_set_keyboard_input_timeout
0001:0000d986  _rl_stuff_char
0001:0000d9fd  _rl_execute_next
0001:0000da16  _rl_clear_pending_input
0001:0000da31  __rl_input_available
0001:0000da79  __rl_input_queued
0001:0000daa7* _rl_getc
0001:0000dd3e  _rl_read_key
0001:0000defa  __rl_insert_typein
0002:00000e54* _waiting_char
0002:00000e50* _rl_getc_function
0002:00004630  _rl_event_hook
Module: U:\extras\lib\libreadline.lib(rltty.obj)
0001:0000dfa0* _rl_tty_unset_default_bindings
0001:0000e03d  __rl_restore_tty_signals
0001:0000e0b2  __rl_disable_tty_signals
0001:0000e17f* _rltty_set_default_bindings
0001:0000e1ed  _rl_tty_set_default_bindings
0001:0000e1f6* _rl_stop_output
0001:0000e21d  _rl_restart_output
0001:0000e244* _rl_deprep_terminal
0001:0000e2c9  _rl_prep_terminal
0002:00000e60  _rl_prep_term_function
0002:00000e64  _rl_deprep_term_function
Module: U:\extras\lib\libreadline.lib(histfile.obj)
0001:0000e8f2  _write_history
0001:0000e90c* _append_history
0001:0000e920  _history_truncate_file
0001:0000ebcb* _read_history_range
0001:0000ef1d  _read_history
0002:00004930* _history_write_timestamps
Module: U:\extras\lib\libreadline.lib(keymaps.obj)
0001:0000ef40* _rl_discard_keymap
0001:0000efa0* _rl_free_keymap
0001:0000efbf  _rl_make_bare_keymap
0001:0000efec* _rl_make_keymap
0001:0000f03b* _rl_copy_keymap
0002:00000e70  _emacs_standard_keymap
0002:00001e90  _emacs_ctlx_keymap
0002:00001680  _emacs_meta_keymap
0002:000026a0  _vi_movement_keymap
0002:00002eb0  _vi_insertion_keymap
Module: U:\tmp\ldconv_libgcc_so_d_a_19c252885a351afc80.lib(emx-ctordtor.obj)
0001:0000f070  ___ctordtorInit
0001:0000f0a4  ___ctordtorTerm
Module: U:\extras\lib\libreadline.lib(xmalloc.obj)
0001:0000f12f  _xrealloc
0001:0000f182  _xmalloc
Module: U:\extras\lib\libreadline.lib(xfree.obj)
0001:0000f1c0  _xfree
Module: U:\extras\lib\libreadline.lib(histexpand.obj)
0002:000057b0+ _history_inhibit_expansion_function
0001:0000f75c* _history_tokenize
0001:0000f80c  _history_arg_extract
0001:0000f9c2* _get_history_event
0001:0000fde1* _history_expand
0002:00003738* _history_word_delimiters
0002:00003730* _history_expansion_char
0002:00003731* _history_subst_char
0002:00003734* _history_no_expand_chars
0002:00004950  _history_comment_char
0002:00004954* _history_quotes_inhibit_expansion
Module: U:\extras\lib\libreadline.lib(util.obj)
0001:00011580  __rl_null_function
0001:00011587* __rl_digit_p
0001:0001159b* __rl_digit_value
0001:000115a6* __rl_lowercase_p
0001:000115d7* __rl_pure_alphabetic
0001:00011606* __rl_to_lower
0001:00011638* __rl_to_upper
0001:0001166a* __rl_uppercase_p
0001:0001169b* __rl_trclose
0001:000116d2* __rl_tropen
0001:0001173a* __rl_trace
0001:00011794* __rl_savestring
0001:000117c7* _rl_free
0001:000117dc  __rl_qsort_string_compare
0001:000117f8  __rl_strindex
0001:00011874  __rl_errmsg
0001:000118e3  __rl_ttymsg
0001:00011959  _rl_tilde_expand
0001:00011a97  _rl_copy_text
0001:00011ae3  _rl_extend_line_buffer
0001:00011b2d  _rl_tty_status
0001:00011b3c  __rl_abort_internal
0001:00011b96  _rl_abort
0001:00011ba8  _rl_alphabetic
0002:000049d0* __rl_allow_pathname_alphabetic_chars
Module: U:\extras\lib\libreadline.lib(tilde.obj)
0001:00011c9d* _tilde_expand_word
0001:00011e55  _tilde_expand
0002:00003740* _tilde_additional_prefixes
0002:00003744* _tilde_additional_suffixes
0002:000049f0* _tilde_expansion_preexpansion_hook
0002:000049f4* _tilde_expansion_failure_hook
Module: U:\extras\lib\libreadline.lib(terminal.obj)
0002:000057c0  __rl_screenheight
0002:000057d0  __rl_screenwidth
0002:000057e0+ __rl_term_backspace
0002:000057f0  __rl_screenchars
0002:00005800  __rl_term_clreol
0002:00005810  __rl_term_cr
0002:00005820  __rl_term_clrpag
0002:00005830  __rl_term_IC
0002:00005840  __rl_term_ic
0002:00005850  __rl_term_ei
0002:00005860  __rl_term_im
0002:00005870  __rl_term_DC
0002:00005880  __rl_term_dc
0002:00005890  __rl_term_up
0002:000058a0+ __rl_term_forward_char
0002:000058b0+ __rl_term_pc
0002:000058c0  __rl_enable_keypad
0002:000058d0+ __rl_term_goto
0002:000058e0+ __rl_term_ip
0001:000121b0* _rl_get_screen_size
0001:000121d3* __rl_set_cursor
0001:000123b1  __rl_output_character_function
0001:0001223c  __rl_control_keypad
0001:00012277  __rl_enable_meta_key
0001:000122aa  _rl_ding
0001:0001231e  _rl_crlf
0001:0001233d  __rl_backspace
0001:000123cd  __rl_output_some_chars
0001:000123f8* _rl_get_termcap
0001:00012517* __rl_get_screen_size
0001:000126e7  __rl_init_terminal_io
0001:00012b55* _rl_reset_terminal
0001:00012b7e* __rl_set_screen_size
0001:00012bf4* _rl_set_screen_size
0001:00012bfd  _rl_resize_terminal
0001:00012c4d* _rl_reset_screen_size
0002:00003760  __rl_term_autowrap
0002:00003764  __rl_enable_meta
0002:00004a00* _rl_prefer_env_winsize
0002:00004a04  __rl_terminal_can_insert
Module: U:\extras\lib\libreadline.lib(signals.obj)
0001:00012dc0* _rl_echo_signal_char
0001:00012e9c* __rl_release_sigwinch
0001:00012ed5  __rl_release_sigint
0001:00012f0f* __rl_block_sigwinch
0001:00012f75  __rl_block_sigint
0001:00012fda* _rl_free_line_state
0001:00013005  _rl_clear_signals
0001:00013137* _rl_cleanup_after_signal
0001:0001322c  _rl_set_signals
0001:00013488* _rl_reset_after_signal
0001:0001362b  __rl_signal_handler
0002:00003770  _rl_catch_signals
0002:00003774  _rl_catch_sigwinch
0002:00004b58* __rl_echoctl
0002:00004b5c  __rl_intr_char
0002:00004b64  __rl_susp_char
0002:00004b60  __rl_quit_char
0002:00004b50  __rl_interrupt_immediately
0002:00004b54  __rl_caught_signal
Module: U:\extras\lib\libreadline.lib(undo.obj)
0001:00013650* __rl_fix_last_undo_of_type
0001:00013683  _rl_do_undo
0001:00013879  _rl_undo_command
0001:000138ad  _rl_revert_line
0001:000138f4  _rl_free_undo_list
0001:00013960  _rl_add_undo
0001:00013999  _rl_end_undo_group
0001:000139ce  _rl_begin_undo_group
0001:00013a03  _rl_modifying
0001:00013a7e* __rl_copy_undo_entry
0001:00013af8* __rl_copy_undo_list
0002:00004ca8  _rl_undo_list
0002:00004ca0  __rl_doing_an_undo
0002:00004ca4  __rl_undo_group_level
Module: U:\extras\lib\libreadline.lib(macro.obj)
0001:00013b50* __rl_push_executing_macro
0001:00013b83  __rl_with_macro_input
0001:00013bac* _rl_push_macro_input
0001:00013bb5  _rl_call_last_kbd_macro
0001:00013c44  _rl_end_kbd_macro
0001:00013c9c  _rl_start_kbd_macro
0001:00013d19  __rl_kill_kbd_macro
0001:00013d7f  __rl_pop_executing_macro
0001:00013ded  __rl_next_macro_key
0001:00013e57  __rl_add_macro_char
0002:00004cb0  _rl_executing_macro
Module: U:\extras\lib\libreadline.lib(misc.obj)
0002:000058f0  __rl_argcxt
0001:00013ee0  __rl_reset_argument
0001:00013f0d  _rl_emacs_editing_mode
0001:00013f32  __rl_set_insert_mode
0001:00013f3f  _rl_overwrite_mode
0001:00013f68  _rl_vi_editing_mode
0001:00013f99  _rl_maybe_save_line
0001:00014011* _rl_replace_from_history
0001:00014068  __rl_revert_all_lines
0001:0001418f  __rl_free_history_entry
0001:000141cd  __rl_free_saved_history_line
0001:000141f2  _rl_maybe_unsave_line
0001:0001424a  __rl_start_using_history
0001:00014272  _rl_maybe_replace_line
0001:000142d5  _rl_get_previous_history
0001:00014404  _rl_get_next_history
0001:0001452b  _rl_beginning_of_history
0001:0001454d  _rl_end_of_history
0001:00014566* _rl_discard_argument
0001:000145a2  __rl_arg_overflow
0001:00014601  __rl_arg_getchar
0001:00014638* __rl_arg_dispatch
0001:0001489d  _rl_universal_argument
0001:000147cd  __rl_arg_callback
0001:0001487c* __rl_arg_init
0001:000148c9  _rl_digit_argument
0002:00003780  __rl_history_saved_point
0002:00004d14  __rl_saved_line_for_history
0002:00004d10  __rl_history_preserve_point
Module: U:\extras\lib\libreadline.lib(vi_mode.obj)
0001:00014930  __rl_vi_initialize_line
0001:00014954  __rl_vi_reset_last
0001:00014981  __rl_vi_set_last
0001:0001499e* _rl_vi_start_inserting
0001:000149cc  _rl_vi_fWord
0001:00014a76  _rl_vi_bWord
0001:00014b38  _rl_vi_eWord
0001:00014c82  _rl_vi_fword
0001:00014dea  _rl_vi_bword
0001:00015045  _rl_vi_eword
0001:000151f5  _rl_vi_append_mode
0001:00015240  _rl_vi_insertion_mode
0001:00015259  _rl_vi_insert_mode
0001:0001528d  _rl_vi_check
0001:000152b1* _rl_vi_bracktype
0001:0001534c  _rl_vi_goto_mark
0001:000153d4  _rl_vi_set_mark
0001:0001541e  _rl_vi_end_word
0001:0001547a  _rl_vi_next_word
0001:000154ec  _rl_vi_prev_word
0001:0001555c  _rl_vi_replace
0001:000156a6  _rl_vi_overstrike
0001:000155fa  _rl_vi_overstrike_delete
0001:00016d21  _rl_vi_movement_mode
0001:000155e0  _rl_vi_eof_maybe
0001:000156ec  _rl_vi_match
0001:00015839  _rl_vi_char_search
0001:000159fe  _rl_vi_back_to_indent
0001:00015a62  _rl_vi_first_print
0001:00015a72  _rl_vi_insert_beg
0001:00015abe  _rl_vi_delete
0001:00015b3d  _rl_vi_rubout
0001:00015c2d  _rl_vi_change_char
0001:00015d0f  _rl_vi_change_case
0001:00015eab  __rl_vi_textmod_command
0001:00016653* _rl_vi_domove
0001:0001669a  _rl_vi_yank_to
0001:00016753  _rl_vi_change_to
0001:00016826  _rl_vi_subst
0001:00016866  _rl_vi_delete_to
0001:00016939  __rl_vi_domove_callback
0001:0001696e  _rl_vi_column
0001:000169a2  _rl_vi_append_eol
0001:00016a03  _rl_vi_redo
0001:00016b2f  _rl_vi_put
0001:00016ba9  _rl_vi_arg_digit
0001:00016c93  __rl_vi_done_inserting
0001:00016d77  _rl_vi_tilde_expand
0001:00016dc3  _rl_vi_complete
0001:00016eb0  _rl_vi_search
0001:00016f0e  _rl_vi_search_again
0001:00016f4c  _rl_vi_fetch_history
0001:00016fbb  _rl_vi_yank_arg
0001:00016ffd  _rl_vi_undo
0002:00003790  __rl_vi_last_command
0002:00004d20  __rl_vimvcxt
Module: U:\extras\lib\libreadline.lib(funmap.obj)
0002:00005900  _funmap
0002:00005910+ _funmap_program_specific_entry_start
0001:00017010  _rl_add_funmap_entry
0001:0001709a  _rl_initialize_funmap
0001:000170f0  _rl_funmap_names
Module: U:\extras\lib\libreadline.lib(nls.obj)
0001:00017dec  __rl_init_eightbit
Module: U:\extras\lib\libreadline.lib(shell.obj)
0001:00017ef0  _sh_unset_nodelay_mode
0001:00017f47  _sh_get_home_dir
0001:00017f67  _sh_get_env_value
0001:00017f84  _sh_set_lines_and_columns
0001:0001801e  _sh_single_quote
Module: U:\extras\lib\ncurses.lib(lib_tputs.obj)
0001:000184f0* __nc_outch
0001:00018090  _tputs
0001:000183f0* _delay_output
0001:000184c0  __nc_flush
0001:00018550  _putp
0002:00004eb0  _PC
0002:00004eb2  _ospeed
0002:00004eb4* __nc_nulls_sent
Module: U:\extras\lib\ncurses.lib(lib_tgoto.obj)
0001:00018580  _tgoto
Module: U:\extras\lib\libreadline.lib(callback.obj)
0002:00005920+ _rl_linefunc
0001:000185a0* __rl_callback_data_dispose
0001:000185ac  __rl_callback_data_alloc
0001:000185d3* _rl_callback_handler_remove
0001:000186be* _rl_callback_read_char
0001:00018a0e* _rl_callback_handler_install
0002:00004ec0  __rl_callback_func
0002:00004ec4  __rl_callback_data
Module: U:\extras\lib\libreadline.lib(kill.obj)
0001:00018a40* _rl_set_retained_kills
0001:00018b2b  _rl_yank_last_arg
0001:00018bf2  _rl_yank_nth_arg
0001:00018c06  _rl_yank
0001:00018c48  _rl_yank_pop
0001:00018fc5  _rl_copy_backward_word
0001:00018fe5  _rl_copy_forward_word
0001:00019005  _rl_copy_region_to_kill
0001:00019013  _rl_kill_text
0001:0001905f  _rl_unix_line_discard
0001:000190ac  _rl_unix_filename_rubout
0001:000191b4  _rl_unix_word_rubout
0001:000192cc  _rl_kill_full_line
0001:00019309  _rl_backward_kill_word
0001:00019368  _rl_kill_word
0001:000193cc  _rl_kill_region
0001:0001940c  _rl_kill_line
0001:00019473  _rl_backward_kill_line
Module: U:\extras\lib\libreadline.lib(isearch.obj)
0001:000195f0* __rl_isearch_dispatch
0001:0001a166  _rl_reverse_search_history
0001:0001a154  _rl_forward_search_history
0001:00019d05  __rl_scxt_dispose
0001:00019e51  __rl_search_getchar
0001:00019e72  __rl_isearch_callback
0001:00019ead  __rl_scxt_alloc
0002:00004f84  __rl_iscxt
0002:00004f80  __rl_isearch_terminators
Module: U:\extras\lib\libreadline.lib(parens.obj)
0001:0001a180* _rl_set_paren_blink_timeout
0001:0001a197* _rl_insert_close
0001:0001a3a1  __rl_enable_paren_matching
0002:000037c0  _rl_blink_matching_paren
Module: U:\extras\lib\libreadline.lib(mbutil.obj)
0001:0001a460* __rl_find_next_mbchar
0001:0001a46b* __rl_find_prev_mbchar
0002:000037d0  _rl_byte_oriented
Module: U:\extras\lib\libreadline.lib(search.obj)
0001:0001a6f6  _rl_history_search_backward
0001:0001a759  _rl_history_search_forward
0001:0001a871  _rl_noninc_reverse_search_again
0001:0001a8a1  _rl_noninc_forward_search_again
0001:0001aa80  __rl_nsearch_callback
0001:0001ac15  _rl_noninc_reverse_search
0001:0001ac35  _rl_noninc_forward_search
0002:00004fb0  __rl_nscxt
Module: U:\tmp\ldconv_libgcc_so_d_a_19c252885a351afc80.lib(emx-eh.obj)
0001:0001ac60  ___ehInit
0001:0001ac96* ___ehTerm
Module: U:\extras\lib\libreadline.lib(histsearch.obj)
0001:0001ae8b  _history_search_prefix
0001:0001aea2  _history_search
0001:0001aeb6* _history_search_pos
0002:00005040  _history_search_delimiter_chars
Module: U:\extras\lib\ncurses.lib(lib_termcap.obj)
0001:0001af20  _tgetent
0001:0001b430  _tgetstr
0001:0001b530  _tgetflag
0001:0001b5b0  _tgetnum
0002:00005050  _UP
0002:00005054  _BC
Module: U:\extras\lib\ncurses.lib(lib_cur_term.obj)
0001:0001b640  _set_curterm
0001:0001b6a0  _del_curterm
0002:000050c0  _cur_term
Module: U:\extras\lib\ncurses.lib(lib_data.obj)
0002:000050d0* _stdscr
0002:000050d4* _curscr
0002:000050d8* _newscr
0002:000050dc* __nc_screen_chain
0002:000050e0  _SP
Module: U:\extras\lib\ncurses.lib(lib_napms.obj)
0001:0001b700  _napms
Module: U:\extras\lib\ncurses.lib(lib_baudrate.obj)
0001:0001b7f0  __nc_baudrate
0001:0001b840  __nc_ospeed
0001:0001b880  _baudrate
Module: U:\extras\lib\ncurses.lib(lib_tparm.obj)
0001:0001b8e0* __nc_tparm_analyze
0001:0001bc10  _tparm
0002:00005110* __nc_tparm_err
Module: U:\extras\lib\ncurses.lib(lib_setup.obj)
0001:0001cf40  __nc_setupterm
0001:0001d3e0* _use_env
0001:0001d3f0* __nc_get_locale
0001:0001d420* __nc_unicode_locale
0001:0001d490* __nc_locale_breaks_acs
0001:0001d5f0* _setupterm
0002:00003860* _ttytype
0002:00005300  _LINES
0002:00005304  _COLS
0002:00005308* _TABSIZE
Module: U:\extras\lib\ncurses.lib(trim_sgr0.obj)
0001:0001d760  __nc_trim_sgr0
Module: U:\extras\lib\ncurses.lib(codes.obj)
0001:0001e2c0  _boolcodes
0001:0001e400  _numcodes
0001:0001e980  _strcodes
Module: U:\extras\lib\ncurses.lib(free_ttype.obj)
0001:0001f000  __nc_free_termtype
0001:0001f0c0* _use_extended_names
0002:00003980  __nc_user_definable
Module: U:\extras\lib\ncurses.lib(doalloc.obj)
0001:0001f0e0  __nc_doalloc
Module: U:\extras\lib\ncurses.lib(comp_error.obj)
0001:0001f170  __nc_warning
0001:0001f280  __nc_err_abort
0001:0001f390  __nc_syserr_abort
0001:0001f4a0* __nc_get_source
0001:0001f4b0* __nc_set_source
0001:0001f4c0  __nc_set_type
0001:0001f520  __nc_get_type
0002:00005310  __nc_suppress_warnings
0002:00005314  __nc_curr_line
0002:00005318  __nc_curr_col
Module: U:\extras\lib\ncurses.lib(read_entry.obj)
0001:0001f550* __nc_read_termtype
0001:0001ffb0* __nc_read_file_entry
0001:00020060  __nc_read_entry
Module: U:\extras\lib\ncurses.lib(fallback.obj)
0001:00020330  __nc_fallback
Module: U:\extras\lib\ncurses.lib(lib_ttyflags.obj)
0001:00020340* __nc_get_tty_mode
0001:000203c0  __nc_set_tty_mode
0001:00020440* _def_shell_mode
0001:000204c0  _def_prog_mode
0001:00020540* _reset_prog_mode
0001:000205f0* _reset_shell_mode
0001:000206c0* _savetty
0001:00020740* _resetty
Module: U:\extras\lib\ncurses.lib(name_match.obj)
0001:000207c0  __nc_name_match
0001:000208b0  __nc_first_name
Module: U:\extras\lib\ncurses.lib(getenv_num.obj)
0001:00020920  __nc_getenv_num
Module: U:\extras\lib\ncurses.lib(comp_parse.obj)
0001:00020980* __nc_delink_entry
0001:00020a30* __nc_read_entry_source
0001:00020c20* __nc_resolve_uses2
0001:00022520* __nc_free_entries
0001:00022550  __nc_free_entry
0001:00022580* __nc_entry_match
0001:00022720* __nc_resolve_uses
0002:00003990* __nc_check_termtype2
0002:00003994* __nc_check_termtype
0002:00005380  __nc_head
0002:00005384* __nc_tail
Module: U:\tmp\ldconv_libgcc_a_19c252885a341db3d0.lib(_alloca.obj)
0001:00022760  __alloca
Module: U:\extras\lib\ncurses.lib(access.obj)
0001:000227a0* __nc_rootname
0001:00022840* __nc_is_abs_path
0001:00022880  __nc_pathlast
0001:000228d0* __nc_basename
0001:00022920  __nc_access
0001:000229f0  __nc_is_dir_path
0001:00022a40* __nc_is_file_path
Module: U:\extras\lib\ncurses.lib(db_iterator.obj)
0001:00022ae0  __nc_next_db
0001:00022c20* __nc_tic_dir
0001:00022c70* __nc_keep_tic_dir
0001:00022cc0  __nc_last_db
0001:00022d00* __nc_first_db
Module: U:\extras\lib\ncurses.lib(setbuf.obj)
0001:00022e10  __nc_set_buffer
Module: U:\extras\lib\ncurses.lib(lib_options.obj)
0001:00022ed0* _curs_set
0001:00022f90* _idlok
0001:00022ff0* _idcok
0001:00023040* _halfdelay
0001:00023090* _nodelay
0001:000230c0* _notimeout
0001:000230e0* _wtimeout
0001:00023100* _keypad
0001:00023190* _meta
0001:00023200* _typeahead
0001:00023220* _has_key
0001:000232a0  __nc_keypad
Module: U:\extras\lib\ncurses.lib(comp_scan.obj)
0001:00023620  __nc_get_token
0001:00024420  __nc_panic_mode
0001:00023f40* __nc_trans_string
0001:00024440  __nc_reset_input
0001:000244a0  __nc_push_token
0002:000053e0  __nc_syntax
0002:000053e4* __nc_curr_file_pos
0002:000053e8  __nc_comment_start
0002:000053ec  __nc_comment_end
0002:000053f0  __nc_start_line
0002:000053f4  __nc_curr_token
0002:00005400* __nc_disable_period
Module: U:\extras\lib\ncurses.lib(parse_entry.obj)
0001:00025190  __nc_parse_entry
0001:00025920* __nc_capcmp
Module: U:\extras\lib\ncurses.lib(alloc_entry.obj)
0001:00027100  __nc_wrap_entry
0001:00027670  __nc_merge_entry
0001:00027770  __nc_init_entry
0001:00027890  __nc_copy_entry
0001:00027900  __nc_save_str
Module: U:\extras\lib\ncurses.lib(alloc_ttype.obj)
0001:000279a0  __nc_align_termtype
0001:00027c80  __nc_copy_termtype
Module: U:\extras\lib\ncurses.lib(home_terminfo.obj)
0001:00028960  __nc_home_terminfo
Module: U:\extras\lib\ncurses.lib(lib_has_cap.obj)
0001:000289f0  _has_ic
0001:00028a60  _has_il
Module: U:\extras\lib\ncurses.lib(lib_raw.obj)
0001:00028ab0* _raw
0001:00028b70  _cbreak
0001:00028c20* _qiflush
0001:00028c80* _noraw
0001:00028d40* _nocbreak
0001:00028de0* _noqiflush
0001:00028e40* _intrflush
Module: U:\extras\lib\ncurses.lib(init_keytry.obj)
0001:00028ec0  __nc_init_keytry
0002:000039c0* __nc_tinfo_fkeys
Module: U:\extras\lib\ncurses.lib(unctrl.obj)
0001:00029720  _unctrl
Module: U:\extras\lib\ncurses.lib(lib_trace.obj)
0002:00005500  __nc_tracing
Module: U:\extras\lib\ncurses.lib(comp_captab.obj)
0001:0002b840  __nc_info_hash_table
0001:0002e480  __nc_cap_hash_table
0001:0002f4a0  __nc_capalias_table
0001:0002f6e0  __nc_infoalias_table
0001:0002f740  __nc_get_table
0001:0002f760* __nc_get_hash_table
Module: U:\extras\lib\ncurses.lib(comp_hash.obj)
0001:0002f780  __nc_find_entry
0001:0002f820  __nc_find_type_entry
Module: U:\extras\lib\ncurses.lib(captoinfo.obj)
0001:0002f960  __nc_captoinfo
0001:00030c10* __nc_infotocap
Module: U:\extras\lib\ncurses.lib(strings.obj)
0001:000335e0  __nc_str_init
0001:00033610* __nc_str_null
0001:00033640* __nc_str_copy
0001:00033670  __nc_safe_strcat
0001:000336e0* __nc_safe_strcpy
Module: U:\extras\lib\ncurses.lib(visbuf.obj)
0001:00033770* __nc_visbuf2
0001:00033810  __nc_visbuf
0001:00033830* __nc_visbufn
Module: U:\extras\lib\ncurses.lib(names.obj)
0001:00033ac0* _boolnames
0001:00033e60  _boolfnames
0001:00033fe0* _numnames
0001:000342e0  _numfnames
0001:00034b60  _strnames
0001:000365a0  _strfnames
Module: U:\extras\lib\ncurses.lib(key_defined.obj)
0001:00036cb0  _key_defined
Module: U:\extras\lib\ncurses.lib(add_tries.obj)
0001:00036cf0  __nc_add_to_try


                        +----------------------+
                        |   Imported Symbols   |
                        +----------------------+

Symbol                              Module
======                              ======

___libc_ForkRegisterModule          libc065
___init_dll                         libc065
___libc_Back_termDll                libc065
___libc_ForkDeregisterModule        libc065
__atfork_callback                   libc065
__Py_NoneStruct                     python27
_PyArg_ParseTuple                   python27
_PyOS_snprintf                      python27
_PyCallable_Check                   python27
_PyExc_TypeError                    python27
_PyErr_SetString                    python27
_PyString_FromString                python27
_PyGILState_Ensure                  python27
_PyList_New                         python27
_PyList_SetItem                     python27
_PyErr_Clear                        python27
_PyGILState_Release                 python27
_PyObject_CallFunction              python27
_PyInt_AsLong                       python27
_PyErr_Occurred                     python27
_PyErr_NoMemory                     python27
_PyInt_FromLong                     python27
_PyString_AsString                  python27
_PyOS_setsig                        python27
_PyOS_InputHook                     python27
_PyMem_Malloc                       python27
_Py_FatalError                      python27
_PyExc_ValueError                   python27
_PyErr_Format                       python27
__errno                             libc065
_PyExc_IOError                      python27
_PyErr_SetFromErrno                 python27
_Py_InitModule4                     python27
_PyOS_ReadlineFunctionPointer       python27
__CRT_init                          libc065
__CRT_term                          libc065
___libc_GLocaleCtype                libc065
___stdinp                           libc065
___stdoutp                          libc065
__std_free                          libc065
__std_strdup                        libc065
__std_malloc                        libc065
__std_memcpy                        libc065
__std_setjmp                        libc065
__read_kbd                          libc065
__std_sigrelse                      libc065
__std_setlocale                     libc065
__std_strncpy                       libc065
__std_strcmp                        libc065
__std_longjmp                       libc065
__std_getenv                        libc065
___ctordtorInit1                    libc065
___ctordtorTerm1                    libc065
___stderrp                          libc065
__std_strcpy                        libc065
__std_time                          libc065
__std_snprintf                      libc065
__std_atol                          libc065
__std_qsort                         libc065
__std_strncmp                       libc065
__std_lstat                         libc065
__std_access                        libc065
__std_putc                          libc065
_getpwnam                           libc065
__std_stat                          libc065
__std_strrchr                       libc065
__scrsize                           libc065
__std_strchr                        libc065
__std_strpbrk                       libc065
__std_closedir                      libc065
__std_opendir                       libc065
__std_readdir                       libc065
__std_strnicmp                      libc065
__std_setpwent                      libc065
__std_getpwent                      libc065
__std_endpwent                      libc065
__std_fwrite                        libc065
__std_fflush                        libc065
__std_atoi                          libc065
__std_fprintf                       libc065
_getpwuid                           libc065
__std_sigsetjmp                     libc065
__std_fputs                         libc065
__std_vsnprintf                     libc065
__std_sprintf                       libc065
__std_stricmp                       libc065
__std_strcat                        libc065
__std_fputc                         libc065
__std_open                          libc065
__std_close                         libc065
__std_read                          libc065
__std_isatty                        libc065
__std_fileno                        libc065
__std_tcsetattr                     libc065
__std_tcgetattr                     libc065
__std_tcflow                        libc065
__std_write                         libc065
__std_fstat                         libc065
___register_frame_table             gcc473
___deregister_frame                 gcc473
__std_exit                          libc065
__std_realloc                       libc065
__std_fclose                        libc065
__std_getpid                        libc065
__std_unlink                        libc065
__std_fopen                         libc065
__std_vfprintf                      libc065
__std_strcoll                       libc065
__std_siglongjmp                    libc065
__std_sigprocmask                   libc065
__std_sigemptyset                   libc065
__std_sigaddset                     libc065
__std_sigaction                     libc065
__std_sigdelset                     libc065
__std_signal                        libc065
__std_kill                          libc065
__std_fcntl                         libc065
__std_getuid                        libc065
__std_setenv                        libc065
__std_abort                         libc065
__std_select                        libc065
__std_strlen                        libc065
__std_nanosleep                     libc065
__std_cfgetospeed                   libc065
__std_calloc                        libc065
__std_nl_langinfo                   libc065
__std_strstr                        libc065
__std_strncat                       libc065
__std_memset                        libc065
__std_strtol                        libc065
__std_setvbuf                       libc065
__std_ftell                         libc065
__std_fgets                         libc065
__std_setmode                       libc065
__std_sscanf                        libc065


                        +--------------------+
                        |   Libraries Used   |
                        +--------------------+

U:\extras\lib\libreadline.lib
U:\extras\lib\ncurses.lib
U:\tmp\ldconv_python2_7_dll_a_19c252885a341d7550.lib
U:\tmp\ldconv_libgcc_a_19c252885a341db3d0.lib
U:\tmp\ldconv_libgcc_so_d_a_19c252885a351afc80.lib
U:\usr\lib\libc_alias.lib
U:\usr\local473\lib\libc_dll.lib
U:\usr\lib\libend.lib


                        +-----------------------+
                        |   Linker Statistics   |
                        +-----------------------+

Stack size:  0000 (0.)
Memory size:  0003c7b0 (247728.)
Link time: 00:00.13
